:10A000000004FF1F9DA3000073A50000A3A500008E
:10A01000B9A50000BBA50000BDA500000000000020
:10A020000000000000000000BFA50000C1A5000066
:10A0300000000000C3A50000C5A50000C7A50000E2
:10A04000C7A50000C7A50000C7A50000C7A5000060
:10A05000C7A50000C7A50000C7A50000C7A5000050
:10A06000C7A50000C7A50000C7A50000C7A5000040
:10A07000C7A50000C7A50000C7A50000C7A5000030
:10A39000C7A50000C7A50000C7A5000072B60E48FB
:10A3A0000E49886000220023002400250026002793
:10A3B000B846B946BA46BB46BC4609488546094830
:10A3C0008047094880470948804762B6002000213D
:10A3D000074A9047FEE7000000A0000000ED00E003
:10A3E0000004FF1F3DA5000079A4000031A5000076
:10A3F00093A500005FF0FF30334908605FF0FF3045
:10A40000324908605FF0FF30314908605FF0FF308B
:10A41000304908605FF0FF302F4908605FF0FF307F
:10A420002E4908605FF0FF302D4908605FF0FF3073
:10A430002C49086070475FF0FF302B4908605FF0DF
:10A44000FF302A4908605FF0FF30294908605FF05B
:10A45000FF30284908605FF0FF30274908605FF04F
:10A46000FF30264908605FF0FF30254908605FF043
:10A47000FF30244908607047234824490860244875
:10A480002449254A521A884207D004E00B78037009
:10A49000491C401C521E002AF8D1204820490A1AA3
:10A4A00003E000210170401C521E002AF9D11D4812
:10A4B0001D491E4A521A04E00B780370491C401CC7
:10A4C000521E002AF8D1704780E100E084E100E0EC
:10A4D00088E100E08CE100E090E100E094E100E040
:10A4E00098E100E09CE100E080E200E084E200E02E
:10A4F00088E200E08CE200E090E200E094E200E01C
:10A5000098E200E09CE200E000A0000008ED00E01E
:10A51000000000000000000000000000000000003B
:10A52000000000000000FF1FD4A50000D4A500001B
:10A5300080B5FFF75FFFFFF77EFF01BD03480068AE
:10A5400050F4700001490860704700BF88ED00E0DA
:10A550004EF68851CEF20001086840F470000860A1
:10A56000BFF34F8FBFF36F8F4FF00070E1EE100A13
:10A570007047FEE700F00BF8002801D0C046C04647
:10A580000020C046C04600F004F800F003F80120A7
:10A590007047FEE700F000B80746384600F002F8C2
:10A5A000FBE7FEE780B5C046C046024A110018200E
:10A5B000ABBEFBE726000200FEE7FEE7FEE7FEE794
:10A5C000FEE7FEE7FEE7FEE7C046C046FFF7C0FF36
:04A5D000FFF7D0FFC2
:040000050000A5C989
:00000001FF
